:100000000C941E060C94F7270C9424280C94460696
:100010000C9446060C9446060C9446060C94460630
:100020000C9446060C9446060C942C130C9446062D
:100030000C9446060C9446060C9446060C94460610
:100040000C9451280C9446060C943F2C0C94822C52
:100050000C9446060C9446060C9446060C944606F0
:100060000C9446060C9446069018F218D118D41831
:10007000D718DA18DD18E018E318F218EC18241A6B
:10008000261A261A241A261A261A261A261A261A72
:10009000261A261A261A261A261A261A261A261A60
:1000A000AA19261A261A261A261A261A1B19261AD9
:1000B000261A261A261A261A261A261A261A261A40
:1000C000261A261A261A261A261A261AB619B61912
:1000D000B619B619B619B619B619B619B619261A37
:1000E000261A261A261A261A261A1B19B519B51900
:1000F000B519B519261AC319C919CF19D519DB199C
:10010000E119E719ED19F719011A0B1A151A5C19FB
:100110001E19261A261A261A261AAA19261A261A65
:10012000261A261A261A261A261A261AB419B419B5
:10013000B419B419261AC319C919CF19D519DB195D
:10014000E119E719ED19F719011A0B1A151A5C19BB
:100150001E19261A261A261A261AAA19591A591ABF
:10016000591A591A591A591A591A591A591A591AF7
:10017000591A591A591A701B701B701B701B701B6F
:10018000701B9E1AA81AB21ABC1A1A1B241B331B06
:10019000441BCC1CE11CED1CF61C051D2A1D331D47
:1001A0007C1D451D8E2094209A20A120AF20D120B7
:1001B000EF20456E746572206D656E752E2E2E00D3
:1001C000546F67676C6564206D6963726F50504D42
:1001D00000546F67676C656420696E76657274653C
:1001E000642050504D2100546F67676C6564205443
:1001F00058206D7574696E672100546F67676C6570
:10020000642074656C656D65747279210050726F3D
:10021000746F636F6C206572726F72207769746897
:100220002052580054696D656F7574207768656E4B
:1002300020636F6E6E656374696E6720746F205201
:100240005800507265737320616E79206B65792058
:10025000746F2063616E63656C00436F6E6E6563DF
:1002600074696E6720746F2052582C20706F776508
:100270007220757020746865205258202877697440
:10028000682062696E6420706C7567206966206EF4
:100290006F74207573696E6720616C776179732064
:1002A00062696E642900546F67676C656420276912
:1002B0006D6D656469617465206F75747075742700
:1002C00000546F67676C65642027736C61766520E6
:1002D0006D6F64652700546F67676C6564202761E4
:1002E0006C776179732062696E642700546F676769
:1002F0006C65642050504D206368616E6E656C20A3
:100300006C696D69740053657420525353492069B8
:100310006E6A656374696F6E206368616E6E656C8A
:100320002028303D3D64697361626C652900536526
:10033000742050504D206D696E696D756D20737914
:100340006E630053657420626561636F6E20696E31
:1003500074657276616C0053657420626561636FC9
:100360006E2064656C617900536574206265616319
:100370006F6E206672657175656E637920696E2097
:10038000487A3A20303D64697361626C652C205074
:10039000783D504D52206368616E6E656C20782CFC
:1003A0002046783D465253206368616E6E656C202E
:1003B00078005365742050574D2073746F7020641B
:1003C000656C61792028302064697361626C6564B2
:1003D0002C20312D323535203D3D20302E317320FB
:1003E0002D2035306D696E29005365742050504DB5
:1003F0002073746F702064656C61792028302064EC
:10040000697361626C65642C20312D323535203D75
:100410003D20302E3173202D2035306D696E29003E
:10042000536574206661696C736166652064656CF0
:1004300061792028302064697361626C65642C20C6
:10044000312D323535203D3D20302E3173202D2089
:1004500035306D696E29002A2A2A2A2A2A2A2A2A50
:100460002A2A2A2A2A2A2A2A2A2A2A2A2A2A2A2AEC
:100470002A2A2A2A0052582041636B6564202D20C5
:1004800072657665727420737563636573736675E0
:100490006C21002A2A2A2A2A2A2A2A2A2A2A2A2AAD
:1004A0002A2A2A2A2A2A2A2A2A2A2A2A2A2A2A2AAC
:1004B000002A2A2A2A2A2A2A2A2A2A2A2A2A2A2AC6
:1004C0002A2A2A2A2A2A2A2A2A2A2A2A2A2A00528E
:1004D000582041636B6564202D20757064617465DC
:1004E000207375636365737366756C21002A2A2A0D
:1004F0002A2A2A2A2A2A2A2A2A2A2A2A2A2A2A2A5C
:100500002A2A2A2A2A2A2A2A2A2A0056616C696457
:100510002063686F69636573206172653A205B319F
:100520005D2D5B31365D20286368616E6E656C20E1
:10053000312D31362900536574206F7574707574D0
:1005400020666F7220706F727420005B585D2061AE
:10055000626F7274206368616E67657320616E6498
:10056000206578697420525820636F6E6669670051
:100570005B535D20736176652073657474696E6783
:100580007320746F205258005B525D20726576654F
:1005900072742052582073657474696E6773207486
:1005A0006F2064656661756C747300557365206EA9
:1005B000756D62657273205B312D445D20746F2010
:1005C0006564697420706F727473205B452D515D92
:1005D00020666F722073657474696E677300202DD6
:1005E00020726563656976657220636F6E66696700
:1005F000757261746F722C20727820737720000AF4
:100600000A6F70656E4C52536E67200053657420FC
:1006100073657269616C2062617564726174653AB8
:10062000200056616C69642063686F696365733A82
:100630002031202D20342B34202F2032202D203823
:10064000202F2033202D20382B34202F2034202D14
:10065000203132202F2035202D2031322B34202FF5
:100660002036202D20313600536574204368616E9A
:100670006E656C20636F6E6669673A20005365741F
:100680002044617461726174652028302D32293AEA
:10069000200053657420486F70206368616E6E653A
:1006A0006C7320286D61782032342C207365706162
:1006B000726174656420627920636F6D6D61732966
:1006C0002076616C69642076616C75657320312DCC
:1006D0003235353A2000536574206368616E6E656B
:1006E0006C2073706163696E6720287831306B48C5
:1006F0007A293A200053657420524620706F77653E
:10070000722028302D37293A200053657420524634
:10071000206D6167696320286865782920652E67E8
:100720002E20307844454144463030443A2000532E
:1007300065742062617365206672657175656E63AC
:10074000792028696E20487A293A20005B5A5D207A
:10075000656E746572207265636569766572206383
:100760006F6E66696775726174696F6E2075746902
:100770006C79005B465D20646973706C61792061FF
:10078000637475616C206672657175656E63696509
:10079000732075736564005B525D2063616C6375E3
:1007A0006C6174652072616E646F6D206B65792079
:1007B000616E6420686F70206C697374005B495DC2
:1007C000207265696E697469616C697A6520736508
:1007D0007474696E677320746F20736B65746368DB
:1007E0002064656661756C7473005B585D2072658A
:1007F00076657274206368616E67657320616E64EC
:100800002065786974206D656E75005B535D20739B
:100810006176652073657474696E677320746F20E8
:10082000454550524F4D20616E64206578697420B3
:100830006D656E7500557365206E756D62657273BA
:10084000205B302D395D20746F20656469742070E1
:100850006172616D657465727300202D2053797328
:1008600074656D20636F6E66696775726174696F18
:100870006E000A0A6F70656E4C52536E672000510D
:1008800029204F7574707574206265666F726520DB
:100890006C696E6B20283D465329203A2000502970
:1008A00020536C617665206D6F64652028657870D3
:1008B0006572696D656E74616C293A20004F29205C
:1008C00054696D65642042494E44206174207374FC
:1008D000617274757020203A20004E292050504DCE
:1008E000206F7574707574206C696D69746564200F
:1008F000202020203A200044495341424C454400E6
:100900004D292050504D205253534920746F20637D
:1009100068616E6E656C202020203A20004C2920F2
:1009200050504D206D696E696D756D2073796E63E1
:10093000202875732920203A200044495341424C15
:100940004544004B29204661696C736166652062ED
:100950006561636F6E20696E74762E2028312D32AA
:10096000353573293A20004A29204661696C736144
:10097000666520626561636F6E2064656C617920D5
:1009800028302D323535203D3E20313073202D204A
:100990003135306D696E293A200049292046616958
:1009A0006C7361666520626561636F6E206672714B
:1009B0002E203A200048292050574D2073746F7024
:1009C0002064656C6179202020202020203A2000BE
:1009D00047292050504D2073746F702064656C61FE
:1009E00079202020202020203A200046292046611E
:1009F000696C736166652064656C617920202020D4
:100A00002020203A200050574D206368616E6E65AB
:100A10006C200066756E6374696F6E3A2000292041
:100A2000706F72742000506F776572546F776572C3
:100A300000445446205548462033322D62697420C4
:100A400031306368004F70656E4C52536E67525878
:100A5000206D696E6920342F36636800466C7974A6
:100A6000726F6E2F4F72616E6765525820554846FF
:100A70002038636800525820747970653A20004429
:100A8000697361626C656400487A00203D3D200016
:100A900043616C63756C61746564207061636B6540
:100AA0007420696E74657276616C3A200042292068
:100AB0004D6963726F202868616C66292050504D23
:100AC000202020203A00412920496E766572746505
:100AD000642050504D20696E20202020203A0030A4
:100AE00029204D7574652062757A7A657220286DAB
:100AF0006F73746C79293A003929205365726961E2
:100B00006C2062617564726174653A00736D617224
:100B100074506F7274004672536B79005472616E38
:100B200073706172656E740044697361626C6564B0
:100B30000038292054656C656D657472793A2020FF
:100B40002020202020003729204368616E6E656CCC
:100B500020636F6E6669673A202000362920446161
:100B60007461726174652028302D32293A2020206A
:100B700000352920486F70206368616E6E656C7364
:100B80003A2020202020003429204368616E6E65C1
:100B90006C2073706163696E673A202000332920EE
:100BA000524620706F7765722028302D37293A2001
:100BB0002020003229205246206D616769633A2067
:100BC0002020202020202020003129204261736530
:100BD000206672657175656E63793A202020000089
:100BE00000000700020100000304060000000000EE
:100BF00000000001020408102040800102040810D7
:100C00002001020408102004040404040404040263
:100C10000202020202030303030303000000002395
:100C2000002600290000000000250028002B0000FD
:100C3000000000240027002A0000702D11241FBE90
:100C4000CFEFD8E0DEBFCDBF13E0A0E0B1E0EEEE25
:100C5000F0E602C005900D92A83CB107D9F716E066
:100C6000A8ECB3E001C01D92AE38B107E1F71CE07B
:100C7000CCE3DCE004C02297FE010E94792ECA3347
:100C8000D107C9F70E94AC2D0C9475300C9400006C
:100C900080917305813019F482E08093730580910F
:100CA0007305833019F484E0809373050895A89543
:100CB0000895DC01ED91FC910190F081E02D099502
:100CC00008952091740530917505382748E0C901D1
:100CD000880F991F37FF06C09C0151E2252750E17C
:100CE000352701C09C01415091F730937505209341
:100CF0007405089588E38093760580E092ECA1E086
:100D0000B0E08093770590937805A0937905B09330
:100D10007A0587E08093830580EC92E9ADEEB9E136
:100D200080937B0590937C05A0937D05B0937E0511
:100D300085E0809384058DEE9EEFADEABEED809355
:100D40007F0590938005A0938105B0938205E5E827
:100D5000F5E080E090E0863028F4DC01AE54BC4F32
:100D60002C9101C020E0219301968831910599F7DB
:100D700082E080939D058AE080939E05089580EC33
:100D800091EDA8E9BBE18093BB059093BC05A093CE
:100D9000BD05B093BE0580E090E0A0E0B0E5809393
:100DA000BF059093C005A093C105B093C205E3ECC5
:100DB000F5E080E081938F5F8031E1F70895A0E056
:100DC000B0E0E5EEF6E00C94422ED82F0E94A72862
:100DD0006115710581059105C9F30E94E52E1092F8
:100DE0007F05109280051092810510928205C4E063
:100DF000812C912C54018A94C0907F05D09080055D
:100E0000E0908105F0908205FE2CED2CDC2CCC24AA
:100E10000E94E02EA50194010E94212E6C0D7D1DE3
:100E20008E1D9F1D60937F057093800580938105C3
:100E300090938205C15001F7DD2309F450C005E805
:100E400015E0E801A12CB12C62E3C62ED12CE12CD7
:100E5000F12C8881882309F442C0B39419F40E94CC
:100E60007A063DC00E94E02EA70196010E94212E25
:100E7000E1E0E60FA5E8B5E08A2F801B8A1520F493
:100E80008D918E13F9CFE9CF2091840530E0A0E158
:100E9000B7E20E94B92D9B01AC01AE2FB0E00E94D9
:100EA000C82D40907B0550907C0560907D0570902A
:100EB0007E05640D751D861D971D4090BB055090E5
:100EC000BC056090BD057090BE05461657066806C5
:100ED000790618F2E993A39488E1A812BACFCDB7A6
:100EE000DEB7E0E10C945E2E8436910520F4BC015F
:100EF00080E090E017C09C018E3B910528F42A55B4
:100F00003109AAE0B0E00CC0823D910528F4245BD1
:100F10003109A4E6B0E004C02D5C3109A8E5B2E0D7
:100F20000E94B92DA4E6B0E09B01AC010E94C82D3F
:100F3000089590E08C599F4F0E947407089561E0D6
:100F400083E10E94542960E083E10E948D2982E0C0
:100F50008093B00085E08093B10061E083E00E945F
:100F6000542960E083E00E948D290895A4E0B0E058
:100F7000ECEBF7E00C94502E009749F19C0140E017
:100F800050E068E478EE81E090E00E94212E61E07C
:100F900083E129833A834B835C830E948D292981D5
:100FA000822F3A81932F4B81A42F5C81B52F8F3FE5
:100FB0009105A105B10529F020F08FEF90E0A0E0A8
:100FC000B0E08093B3008091B000806107C060E022
:100FD00083E10E948D298091B0008F7E8093B000C4
:100FE0002496E2E00C946C2E60E08CE00E94542980
:100FF00061E08BE00E94542961E08DE00E94542959
:1010000060E082E00E94542961E084E00E9454295B
:10101000089542E050E068E476E080E00E94D7273F
:101020000895E3E0F0E089E080935700E491E670F2
:1010300081E0E63009F080E00895CF93DF93C82F78
:101040000E941108882381F0DFB781E08093720548
:10105000F8940E94570688E180936000C093600076
:10106000C1110E945706DFBFDF91CF9108958F9283
:101070009F92AF92BF92CF92DF92EF92FF92CF9367
:10108000FC01C0A5EC2FE770F0E0E658FC4FA08112
:10109000B0E0C7FF03C024E130E002C02FE030E041
:1010A000FC0197A183E1989FF0011124E25CFE4FBF
:1010B00080809180A280B380A20FB31F20E43FE123
:1010C0004DE750E00E94D32DA50194010E94FF2D11
:1010D0008C2F887149F469017A01E0EDCE0EE7E0CA
:1010E000DE1EE11CF11C1BC0C7FF05C060E47AE8EE
:1010F0008CE29EE004C060E07EEE8AEB9BE069013A
:101100007A01F8EBCF0EFBE0DF1EE11CF11CA5011C
:1011100094010E94FF2DC20ED31EE41EF51EC701CE
:10112000B60169517C4F8F4F9F4F28EE33E040E06E
:1011300050E00E94FF2DA8EEB3E00E94C82DCF9191
:10114000FF90EF90DF90CF90BF90AF909F908F90E7
:1011500008958F3F910551F048F0811522E09207E4
:1011600038F08115934030F482E0089580E00895CE
:1011700081E0089583E00895A0E0B0E0E2ECF8E0BB
:101180000C944B2EEB018A01B82FB695A0E0288174
:101190003981F80120832A813B8121832C813D8183
:1011A00022832E813F812383688179814A815B81FB
:1011B0002C813D81EE81FF819F2F9295990F990F90
:1011C000907C272F2370922B252F2370220F220F24
:1011D000922B232F23702295207F922BF80194834A
:1011E0000B5F1F4F2896AF5FBA1788F680FF24C0A9
:1011F000888199810E94A908D82E8A819B810E94AA
:10120000A908E82E8C819D810E94A908F82E8E8164
:101210009F810E94A908F0E4DF9EA001112490E1C3
:10122000E99E90011124242B282BE4E0FE9EB001BE
:101230001124262BF8012083CDB7DEB7E7E00C940C
:10124000672E803223E0920708F1883E23E0920760
:1012500040F48F519340E4E096958795EA95E1F745
:101260000895803D27E0920718F48C5D934008951F
:10127000883928E0920768F4885C974074E0969576
:1012800087957A95E1F78D509C4F089580E090E026
:1012900008958FEF93E008958C30910540F4A4E019
:1012A000880F991FAA95E1F7885D9C4F0895843FA8
:1012B00023E0920718F484529C4F0895811524E08E
:1012C000920740F48657934FF4E0880F991FFA95E0
:1012D000E1F7089580E998E008959C0136952795F7
:1012E00025753575821B930B9C012373337396957B
:1012F00087959695879583739373820F931F9C01AF
:1013000054E0369527955A95E1F7280F391F2F702D
:101310003F7041E051E0249FC001259F900D349F14
:10132000900D1124892F08952D98882319F000001D
:101330002B9A02C000002B9800002D9A00000895FF
:101340002D9A000083B12D98000082958170089538
:10135000CF93DF93D82F5C9A2D985C98C8E08D2F9F
:1013600080780E949409DD0FC150C9F72D98DF9154
:10137000CF9108958F770E94A8090895CF93DF93A6
:10138000D82FC8E08D2F80780E949409DD0FC150BE
:10139000C9F72D98DF91CF910895CF93DF932D98C2
:1013A000C8E080E0D82FDD0F0E94A0098D0FC1504A
:1013B000C9F7DF91CF9108950E94BA090E94CD0923
:1013C0005C9A0895A1E0B0E0E8EEF9E00C94502EAC
:1013D000806869830E94A8096981862F0E94BE09DE
:1013E0005C9A2196E2E00C946C2ECF93C0917F051D
:1013F000C827E82FF0E0EA58FA4F678589E70E948E
:10140000E2096C2F8DE30E94E2096C2F82E40E94B6
:10141000E209CF91089586E20E94DC090895CF93F6
:10142000DF93EC016C818CE10E94E2096D818DE11A
:101430000E94E2096E818EE10E94E2096F8180E2E2
:101440000E94E209688581E20E94E209698582E2E0
:101450000E94E2096A8583E20E94E2096B8584E2C8
:101460000E94E2096C8585E20E94E2096D858AE2AC
:101470000E94E2096E858EE60E94E2096F858FE682
:101480000E94E209688980E70E94E209698981E790
:101490000E94E2096A8982E70E94E209DF91CF9106
:1014A0000895CF92DF92EF92FF92CF93DF936B017B
:1014B0007C01C11488E3D8068CE9E8068CE1F806C3
:1014C00028F5C701B60120E836E948E950E00E9456
:1014D000FF2DE901689760E879E687E69FEF0E94B3
:1014E000DB2D6C0D7D1D8E1D9F1DF2E0660F771F9D
:1014F000881F991FFA95D1F721E732E040E050E0CC
:101500000E94FF2DF22EE32E80E421C0C701B60118
:1015100020E03DE241E351E00E94FF2DE9016897A0
:1015200060E073ED8EEC9EEF0E94DB2D6C0D7D1D57
:101530008E1D9F1D660F771F881F991F21E732E0C0
:1015400040E050E00E94FF2DF22EE32E80E66C2F4B
:101550006F71680F85E70E94E2096E2D86E70E9491
:10156000E2096F2D87E70E94E209DF91CF91FF909A
:10157000EF90DF90CF900895682F8DE60E94E209EA
:1015800008958F929F92AF92BF92CF92DF92EF9287
:10159000FF92CF93DF93D82F83E00E94DC098093E2
:1015A000710584E00E94DC098093700560E086E0AC
:1015B0000E94E20961E087E00E94E2096FE789E0AA
:1015C0000E94E20965E08AE00E94E20962E18BE0A4
:1015D0000E94E20965E18CE00E94E2096DEF8DE076
:1015E0000E94E20960E08EE00E94E209DD2319F02A
:1015F0008BE291E008C020919D0533E1239FC0015B
:101600001124825C9E4F0E940F0A6CE880E30E94C6
:10161000E2096FE082E30E94E20962E483E30E9450
:10162000E20980919E0587FF02C064E101C06AE083
:1016300084E30E94E2096AE285E30E94E2096DE226
:1016400086E30E94E20964ED87E30E94E20960E01C
:1016500088E30E94E20960E089E30E94E209D11177
:1016600009C0C0907F05D0908005E0908105F09082
:10167000820507C0C5E9CC2EC1ECDC2EED2CCEEDE9
:10168000FC2ECAE38F2C9924AA24BB24682D8C2F0E
:101690000E94E209682D85E08C0F0E94E209FE2C71
:1016A000ED2CDC2CCC24CF5FCE3361F76FEF83E4DD
:1016B0000E94E2096FEF84E40E94E2096FEF85E483
:1016C0000E94E2096FEF86E40E94E209DD2311F037
:1016D00066E002C0609183058DE60E94E20960E049
:1016E00089E70E94E209609184058AE70E94E20985
:1016F00060E083E70E94E20960E084E70E94E2097B
:10170000D11109C060917B0570917C0580917D05A8
:1017100090917E0504C060EC72E98DEE99E10E9423
:10172000510ADF91CF91FF90EF90DF90CF90BF9063
:10173000AF909F908F90089561E087E00E94E2094A
:1017400064E28EE70E94E20963E088E00E94E20919
:1017500060E088E00E94E20965E087E00E94E2091B
:1017600062E085E00E94E20983E00E94DC09809348
:10177000710584E00E94DC0980937005089583E080
:101780000E94DC098093710584E00E94DC0980934B
:10179000700561E087E00E94E2096AE070E080E0A5
:1017A00090E00E94CA280E949C0B00000895CF92EE
:1017B000DF92FF920F931F93CF93DF931F92CDB7CA
:1017C000DEB7082F162F8EE399830E94E209F02ED0
:1017D000C02E9981D92E8C2D8F19811738F4F601DE
:1017E00061916F018FE70E94E209F5CF64E085E027
:1017F0000E94E20983E00E94DC098093710584E085
:101800000E94DC09809370050E94A72860936C05F4
:1018100070936D0580936E0590936F0569E087E086
:101820000E94E20981E0809373050F90DF91CF91D0
:101830001F910F91FF90DF90CF9008950F931F930A
:101840000E94D70B80917305813099F40E94A728DC
:1018500000916C0510916D0520916E0530916F051A
:10186000601B710B820B930B603A764881409105A7
:1018700048F380917305813031F46EE971E082EEB6
:1018800095E00E94932A1F910F9108950F931F9343
:1018900080917305823021F41092730581E020C09D
:1018A000809173058130D9F40E94A72800916C05BE
:1018B00010916D0520916E0530916F05601B710BC5
:1018C000820B930B613A76488140910540F061E0CC
:1018D00087E00E94E2091092730582E001C080E077
:1018E0001F910F910895CF93DF93EC014AE050E0F0
:1018F0006D2F70E082EE95E00E94612B6EE282EE29
:1019000095E00E94652ABE0184E0769567958A95E8
:10191000E1F76F7077274AE050E082EE95E00E9491
:10192000612B6EE282EE95E00E94652ABE016F7027
:1019300077274AE050E082EE95E00E94612BDF912C
:10194000CF910895D82FC0E0CD1780F4439A64E674
:1019500070E080E090E00E94CA28439864E670E05E
:1019600080E090E00E94CA28CF5FEECF6CE271E089
:1019700080E090E00E94CA28E6CF0F931F93CF9398
:10198000DF93EC01062F15E0115051F0CE010E94BB
:101990005C30081741F0602FCE010E946430F4CF14
:1019A00082E00E94A20CDF91CF911F910F910895C8
:1019B000A0E0B0E0EEEDFCE00C94422E482E562E56
:1019C000C0E0D0E0612C712CE12CF12C00E010E0A3
:1019D00041100CC06090D40586E4689E300111244B
:1019E00059E1E52EF12C0AEB15E01EC091E04912F9
:1019F0000FC06090D405E6E46E9E30011124FBE137
:101A00006F0E711C49E2E42EF12C06E715E00CC0C4
:101A100082E0481209C028E1622E77247394EE24F4
:101A2000E394F12C03ED15E043018C0E9D1E109202
:101A30007505109274053401A62CA818B12CC301A9
:101A400001966C01AE14BF04A8F4A00EB11E511093
:101A500006C0C3010E945C30F501808305C0F5011A
:101A60006081C3010E94BD0CF50180810E94610666
:101A70003601E2CFC301511018C0C3010E945C308F
:101A8000B82EC6010E945C302B2D30E0322F222769
:101A9000282B80917405909175058217930779F42E
:101AA000C0E0D0E05524539493CF36016091750582
:101AB0000E94BD0C60917405C6010E94BD0CC05E01
:101AC000DE4FC13E92E0D90708F482CF852DCDB715
:101AD000DEB7E0E10C945E2E61E082E00E94D80C5B
:101AE000089560E082E00E94D80C8091D305853093
:101AF00020F01092D3050E946C0D8091D305809345
:101B0000D405089561E080E00E94D80C61E081E096
:101B10000E94D80C089560E080E00E94D80C8823D1
:101B200051F060E081E00E94D80C882321F0809180
:101B30007605883349F00E94BF060E947A0681E04C
:101B40000E94DF060E94820D0895882319F06AEA38
:101B500071E002C06EEA71E082EE95E00E94932A85
:101B60000895FF920F931F93CF93DF9369EC7BE06F
:101B700082EE95E00E943F2A40917B0550917C05C2
:101B800060917D0570917E052AE030E082EE95E05F
:101B90000E94682B63EB7BE082EE95E00E943F2A77
:101BA00040917F055091800560918105709182057B
:101BB00020E130E082EE95E00E94682B6DE97BE049
:101BC00082EE95E00E943F2A4AE050E06091830552
:101BD00082EE95E00E94902B67E87BE082EE95E034
:101BE0000E943F2A4AE050E06091840582EE95E031
:101BF0000E94902B61E77BE082EE95E00E943F2AF5
:101C0000C5E8D5E0F12C8E0188818823A9F0FF205A
:101C100031F061EB71E082EE95E00E94622A21963C
:101C20004AE050E0F801608182EE95E00E94592B75
:101C3000F394F8E1FF12E7CF82EE95E00E946D2A5F
:101C40006BE57BE082EE95E00E943F2A4AE050E09F
:101C500060919D0582EE95E00E94902B66E47BE00A
:101C600082EE95E00E943F2AE0919E05E770F0E049
:101C7000EE0FFF1FEE57FC4F6081718182EE95E001
:101C80000E94932A61E37BE082EE95E00E943F2A66
:101C900080919E058871883069F028F4811113C005
:101CA00068E27BE00CC0803141F0883161F46CE087
:101CB0007BE005C06CE17BE002C066E17BE082EE88
:101CC00095E00E94812A68EF7AE082EE95E00E941A
:101CD0003F2A409177055091780560917905709180
:101CE0007A052AE030E082EE95E00E94682B6FEDE5
:101CF0007AE082EE95E00E943F2A8091BF058071D4
:101D00000E94A50D66EC7AE082EE95E00E943F2AE3
:101D10008091BF0580740E94A50D6DEA7AE082EE85
:101D200095E00E943F2A8091BF0580720E94A50D18
:101D300060E97AE082EE95E00E943F2A86E795E02E
:101D40000E943708AB01BC012AE030E082EE95E04A
:101D50000E944A2B6BE87AE082EE95E00E943F2ACF
:101D600086E795E00E9437089B01AC0160E472E4CD
:101D70008FE090E00E94FF2DBA01A9012AE030E037
:101D800082EE95E00E944A2B68E87AE082EE95E0C8
:101D90000E94812ACDB7DEB7E5E00C94692E8F92C0
:101DA0009F92AF92BF92CF92DF92EF92FF928111FA
:101DB00007C06FE77AE082EE95E00E94812A2FC08B
:101DC00090E00E94740724E630E040E050E00E947A
:101DD000FF2DCA01B9012AE030E040E050E00E9446
:101DE000FF2D49015A016B017C012AE030E0B50169
:101DF000A40182EE95E00E944A2B6EE282EE95E00D
:101E00000E94652A2AE030E0B701A60182EE95E043
:101E10000E944A2B63E782EE95E00E94A52AFF907C
:101E2000EF90DF90CF90BF90AF909F908F900895EC
:101E30001F93CF93DF9365E77AE082EE95E00E94EF
:101E40003F2A80919F05813041F46CE57AE082EE73
:101E500095E00E94812A10E050C0823019F465E4B8
:101E60007AE0F5CF843019F461E37AE0F0CF853081
:101E700091F766E27AE0EBCFC12FD0E0C930D1050F
:101E80000CF441C068E3610F82EE95E00E94652A80
:101E90006EE17AE082EE95E00E943F2ABE016F5F1C
:101EA0007F4F4AE050E082EE95E00E94292B63E1EB
:101EB0007AE082EE95E00E943F2AC156DA4FE9812E
:101EC000E03218F566E07AE082EE95E00E943F2A63
:101ED0008981803130F06DE673E082EE95E00E94FA
:101EE000622A69816F7070E06F5F7F4F4AE050E057
:101EF00082EE95E00E94322B1F5F809148051817F3
:101F000008F4BACF0FC061E3BECFEF70F0E0EE0F80
:101F1000FF1FEE56FC4F6081718182EE95E00E94BA
:101F2000932AEACF6BEE79E082EE95E00E943F2A99
:101F30008091B7050E94CF0E60ED79E082EE95E0CA
:101F40000E943F2A8091B8050E94CF0E65EB79E090
:101F500082EE95E00E943F2A8091B9050E94CF0E43
:101F60006AE979E082EE95E00E943F2A4091AF0550
:101F70005091B0056091B1057091B20541155105C0
:101F80006105710539F12AE030E082EE95E00E94AA
:101F9000682B67E679E082EE95E00E943F2A809107
:101FA000B3050E949907AB01BC012AE030E082EE44
:101FB00095E00E94682B63E479E082EE95E00E9450
:101FC0003F2A4AE050E06091B40582EE95E00E941D
:101FD000902B06C06AE379E082EE95E00E94812AA8
:101FE0006DE179E082EE95E00E943F2A6091B505AF
:101FF0007091B6054AE050E082EE95E00E947A2B9F
:1020000060E079E082EE95E00E943F2A6091AE05A3
:10201000603450F470E06F5F7F4F4AE050E082EE32
:1020200095E00E94322B06C067EF78E082EE95E0E3
:102030000E94812A6AED78E082EE95E00E943F2AB4
:102040008091AD0580FF03C063EB71E002C067EBD8
:1020500071E082EE95E00E94932A6DEB78E082EECB
:1020600095E00E943F2A8091AD0582700E94A50DE7
:102070006EE978E082EE95E00E943F2A8091AD05FE
:1020800084700E94A50D6FE778E082EE95E00E94D3
:102090003F2A8091AD0588700E94A50DDF91CF91F8
:1020A0001F9108950F931F93CF93DF9320914505C0
:1020B0002F3FA9F56FEF75E082EE95E00E943F2A71
:1020C00082E893E00E94730C6EED75E082EE95E07D
:1020D0000E943F2A80914605909147050E94730C0B
:1020E0006BEA75E082EE95E00E94812A68E875E06F
:1020F00082EE95E00E94812A60E775E082EE95E02D
:102100000E94812A6BE475E082EE95E00E94812AAC
:1021100082EE95E00E946D2A0E94180F68C0121688
:102120000CF065C0332727FD30958091480590E07D
:10213000821793070CF45BC066E375E082EE95E0CE
:102140000E943F2A60914505772767FD70954AE018
:1021500050E082EE95E00E94322B6BE075E082EE5B
:1021600095E00E943F2A10E008E280914905181787
:10217000D0F5C12FD0E0CC0FDD1FC65BDA4F288130
:1021800030E080914505992787FD909501972817A4
:10219000390739F56BEB71E082EE95E00E94622A17
:1021A0004AE050E0602F82EE95E00E94592B6FEBE1
:1021B00071E082EE95E00E94622AE981EF70F0E022
:1021C000EE0FFF1FEE56FC4F6081718182EE95E0AD
:1021D0000E94622A63EC71E082EE95E00E94622A1E
:1021E0000F5F1F5FC2CF82EE95E00E946D2ADF91E4
:1021F000CF911F910F910895FF920F931F93CF934B
:10220000DF93C5E8D5E0F12C8E0188818823D1F1D8
:1022100065EC71E082EE95E00E94622A4AE050E0AF
:102220006F2D82EE95E00E94592B62ED71E082EEF7
:1022300095E00E94622A2196F801208130E0A0E119
:10224000B7E20E94B92D9B01AC01A0918405B0E0DA
:102250000E94C82DAB01BC0180917B0590917C054B
:10226000A0917D05B0917E05480F591F6A1F7B1F05
:102270002AE030E082EE95E00E94682BF394F8E1CA
:10228000FF12C2CFCDB7DEB7E5E00C94692E1092F5
:10229000DF0485E6E0EEF4E0DF011D928A95E9F7C0
:1022A0000895CF93C82F8F3719F0883009F045C0B3
:1022B000E091DF04EE23D9F1E150E093DF04F0E098
:1022C000E052FB4F10826DE070E082EE95E00E94DC
:1022D0005906C0E08091DF04C81760F4EC2FF0E0ED
:1022E000E052FB4F608170E082EE95E00E9459065B
:1022F000CF5FF0CF60E270E082EE95E00E94590679
:102300006DE070E082EE95E00E945906C0E0809199
:10231000DF04C81778F5EC2FF0E0E052FB4F608146
:1023200070E082EE95E00E945906CF5FF0CF67E043
:1023300082EE95E00E94652A1DC08B3119F40E943F
:1023400047111AC08D30C1F08A30B1F08091DF049E
:10235000843668F76C2F70E082EE95E00E94590693
:10236000E091DF0481E08E0F8093DF04F0E0E05223
:10237000FB4FC08380E001C081E0CF910895CF93EF
:10238000C82F0E94A7286093C8047093C904809343
:10239000CA049093CB04C093DD04CC2329F040E021
:1023A00051EE60E070E004C040E855E260E070E0AB
:1023B00082EE95E00E94EF2CCF9108959091CC048D
:1023C000492F4F7050E0BA016F5F7F4F292F30E0E7
:1023D000E4E035952795EA95E1F76217730759F020
:1023E000FA01E353FB4F808381E0890F8F70907F68
:1023F000892B8093CC0408956EE770E082EE95E01F
:102400000E9459060895A3E1B1E0E9E0F2E10C94DD
:10241000432EE5E8F5E0712C8191882321F0739437
:1024200028E17212F9CF66ED71E082EE95E00E942C
:10243000932A4AE050E0672D82EE95E00E94902BAF
:1024400080E00E94C10A0E949C0B8E010E5F1F4F0C
:10245000C12CD12C7601C39466246A945C2C0E9412
:102460009B284B015C012091840530E0A0E1B7E29C
:102470000E94B92D9B01AC01C701B6010E94DB2D62
:1024800020917B0530917C0540917D0550917E0522
:10249000620F731F841F951F2091BB053091BC05EF
:1024A0004091BD055091BE052617370748075907CB
:1024B00018F4F801608225C08C2D0E94F50961E0B6
:1024C00070E080E090E00E94CA28F80110820E942B
:1024D0009B28681979098A099B09643F7140810525
:1024E000910540F40E940B0AF8019081981778F743
:1024F0008083EDCF50FE03C04298439A02C0429AB7
:1025000043982FEFC21AD20AE20AF20A0F5F1F4F56
:102510008FEFC816D104E104F10409F09FCFCE017A
:102520009395FC01D82E7FEF68EC2E2F281B2715E2
:1025300010F051E056C0DE01129651E02FEF41E05D
:102540003D91321710F0322F01C0452F5F5F5F3F82
:1025500011F0232FF5CF4193242F30E0A1E0B0E01C
:10256000AC0FBD1FA20FB31F5C93413079F0DE01A9
:10257000A20FB31F5C93423049F0AFEFBFEFAC0F37
:10258000BD1FA20FB31F6C934E3F78F6A2E0B0E0E0
:10259000AC0FBD1FA20FB31F7C934D3F30F6A3E0DD
:1025A000B0E0AC0FBD1FA20FB31F6C93BECF452F81
:1025B000242F30E0FC01E20FF31F6081AFEFB0E0A9
:1025C000AC0FBD1FA20FB31F2C91621748F44150EE
:1025D000DC01A40FB11D2C9120836C934111E8CF35
:1025E0005F5F571520F3372D369520E0231770F4E1
:1025F000DC01A20FB11D4C91522F530FFC01E50FCE
:10260000F11D50815C9340832E5FF0CFF5E8EF2EF3
:10261000F5E0FF2E8C01802F8D19871598F4F801B5
:10262000C1908F014AE050E06C2D82EE95E00E944F
:10263000592B6CE282EE95E00E94652AF701C19267
:102640007F01E9CF82EE95E00E946D2A81E0CD5EA8
:10265000DE4FEFE00C945F2E1F920F920FB60F9299
:1026600011241F932F933F934F935F936F937F9307
:102670008F939F93AF93BF93CF93DF93EF93FF938A
:10268000C0918600D0918700809187049091880442
:102690002091A904211155C09E01281B390B80915E
:1026A000BF059091C005A091C105B091C20585FDFF
:1026B00002C036952795253C49E03407B8F1409192
:1026C0000A0150E060E070E02CE1B695A79597957F
:1026D00087952A95D1F70097A105B10521F481E0EE
:1026E00090E0A0E0B0E084179507A607B707D8F4FC
:1026F00080910A018F3FB9F040E080910A014817AC
:1027000080F4842F90E0880F991FFC01E757FB4F5E
:1027100020813181FC01E55FFE4F318320834F5FD3
:10272000ECCF1092AA0410920A010BC02D3B82E05C
:10273000380720F080910A018031D8F08FEF809324
:102740000A01D0938804C0938704FF91EF91DF9131
:10275000CF91BF91AF919F918F917F916F915F9139
:102760004F913F912F911F910F900FBE0F901F908F
:10277000189510910A0181E0810F80930A01C90127
:102780000E942109E12FF0E0EE0FFF1FE757FB4FFA
:1027900091838083D6CF83E0809380008AE9809301
:1027A00081008091BF0586FD05C080918100806415
:1027B000809381008FEF9FEF909389008093880032
:1027C00080916F00806280936F0008950E94710D68
:1027D0008091D405843011F41092D40508956F309F
:1027E00018F086958058089589E0689F802D1124FF
:1027F0000895A0E0B0E0EFEFF3E10C944A2EC82F6B
:102800000E94A728009138041091390420913A04BD
:1028100030913B046B017C01C01AD10AE20AF30A31
:102820009701860149E8C41643E1D406E104F104A6
:1028300010F010923C046093380470933904809334
:102840003A0490933B042091A9048FEF820F8230C9
:10285000D8F5E0913C04EE2309F44EC1E13011F4C7
:1028600082E0B8C1E03108F034C181E08E0F80937E
:102870003C04F0E0E757FB4FC083803109F0ACC166
:10288000EBE8F4E0213029F4A181A695A69580819A
:1028900008C080819181A92FA695A695A6959695A9
:1028A0008795A03148F4B0E090E0AA0FBB1FA55F68
:1028B000BE4F11969C938E931092AA04329684E098
:1028C000E939F807F9F688C1233009F005C1E0912C
:1028D0003C04E11104C0CF3009F07EC10DC1E831E4
:1028E00048F481E08E0F80933C04F0E0E857FB4F02
:1028F000C08372C1E83109F0ECC0C111EAC040E008
:1029000050E0ABE0CA01B3E0880F991FBA95E1F738
:10291000A49F9001A59F300D1124F901E757FB4FAB
:102920006081E1817E2F777075956795FC01EE0FD0
:10293000FF1FE55FFE4F71836083F901E657FB4F90
:10294000B081B695B695B695E181FE2FF295FF0F51
:10295000F07E6F2F6B2BE695E695E6957E2F7770D0
:1029600075956795FC01EE0FFF1FE35FFE4F7183C6
:102970006083F901E557FB4FB081B295B695B695E6
:10298000B370C181DC2FDD0FDD0F6D2F6B2BC29576
:10299000C695C695C370E281E170EE0FEE0F7E2FF3
:1029A0007C2B75956795FC01EE0FFF1FE15FFE4FD5
:1029B00071836083F901E357FB4FB081B695E181E4
:1029C000FE2FF795FF27F7956F2F6B2BE6957E2F40
:1029D000777075956795FC01EE0FFF1FEF5EFE4F58
:1029E00071836083F901E257FB4FB081B295BF70EC
:1029F000E181FE2FF295F07F6F2F6B2BE295EF7048
:102A00007E2F777075956795FC01EE0FFF1FED5EC9
:102A1000FE4F71836083F901E157FB4FB081BB1F0B
:102A2000BB27BB1FC181DC2FDD0F6D2F6B2BCC1F94
:102A3000CC27CC1FE281E370EE0F7E2F7C2B7595A7
:102A40006795FC01EE0FFF1FEB5EFE4F7183608305
:102A5000F901EF56FB4FB081B695B695E181FE2F97
:102A6000F295FF0FFF0FF07C6F2F6B2BE695E6952D
:102A70007E2F777075956795FC01EE0FFF1FE95E5D
:102A8000FE4F71836083F901EE56FB4F2081229542
:102A9000269527703181E32FEE0FEE0FEE0F6E2F8C
:102AA000622B732F72957695777075956795FC01FB
:102AB000EE0FFF1FE75EFE4F718360834F5F5F4F36
:102AC0004230510509F01ECF80919F0483FF109280
:102AD000AA0410923C0480C0243009F07DC06091AB
:102AE0003C0461110BC0C83AB1F410927505109204
:102AF000740588EA0E94610681E06CC0613019F4B7
:102B0000C093370404C0623031F4C09336048C2F74
:102B10000E9461065AC0E09136042E2F30E0220F49
:102B2000331F462F50E0C9010296841795073CF0E9
:102B3000633268F7FA01EA57FB4FC083E8CF2D5F95
:102B40003F4F8C2F90E0609174057091750542178E
:102B5000530749F4982F8827862797279093750560
:102B60008093740532C06817790769F5809137043E
:102B7000813049F5E13118F080E180933604F0901E
:102B80003604CAE8D4E000E010E00F15D0F4FE01EE
:102B90003197808190E0982F88272881822B63E0ED
:102BA000969587956A95E1F70E942109F801EE0F45
:102BB000FF1FE55FFE4F918380830F5F1F4F2296BB
:102BC000E4CF1092AA0410923C0480913C04882324
:102BD00019F08F5F80933C04CDB7DEB7E8E00C942A
:102BE000662EE82FF0E0E654FA4FE185E03150F42C
:102BF000F894F0E0EE0FFF1FE55FFE4F80819181BA
:102C000078940895E03121F0E13131F483E101C09D
:102C100082E10E94E929089580E092E00895A2E20D
:102C2000B0E0E5E1F6E10C94402E9E012F5F3F4FAE
:102C300080E1D9011D928A95E9F764E072E082EEA5
:102C400095E029A33AA30E94932A0E94BF0B1D8AF4
:102C50001E8A1F8A188E312C212C00E0812C912C89
:102C6000540170E4472E71EE572E7DE9672E78E10E
:102C7000772EE0E5CE2EE3ECDE2EE12CF12C84EF76
:102C800091E0A0E0B0E08D8F9E8FAF8FB8A380EC75
:102C900091EDA8E9BBE1898F9A8FAB8FBC8F80E45F
:102CA00091EEADE9B8E1898B9A8BAB8BBC8B82EE50
:102CB00095E00E94A72B892B09F4E1C082EE95E0F4
:102CC0000E94D42B9C0133272C32310509F442C0D9
:102CD000ACF42332310509F0ABC019821A821B8291
:102CE0001C821D821E821F82188619861A861B86E8
:102CF0001C861D861E861F86188A60C024343105F6
:102D000029F02335310509F4B2C092C064E482EEA3
:102D100095E00E94652A2AE030E040E451EE6DE93A
:102D200078E182EE95E00E94F32A6CE282EE95E073
:102D30000E94652A2AE030E040EC51ED68E97BE131
:102D400082EE95E00E94F32A6CE282EE95E00E940A
:102D5000A52AADCF0F5F043009F0A9CF29813A81B0
:102D60004B815C81A8EEB3E00E94C82D698B7A8B01
:102D70008B8B9C8B2D813E814F8158850E94C82D65
:102D8000698F7A8F8B8F9C8F29853A854B855C85DF
:102D90002D8F3E8F4F8F58A32D853E854F855889A7
:102DA0000E94C82D6B017C0160323EE473078105EF
:102DB000910530F462E38CE10E94E20900E077CFF4
:102DC000603345E774078105910510F462E2F3CFA3
:102DD00060345CE975078105910510F466E2EBCF7C
:102DE00080E5C81683ECD806E104F10410F462E132
:102DF000E2CF90E6C9169AEED906E104F10410F488
:102E000065E1D9CFA0E7CA16A1E1DA06A1E0EA069A
:102E1000F10410F461E0CFCFB0EACB16B6E8DB06E0
:102E2000B1E0EB06F10410F463E0C5CF65E0C3CF79
:102E300010ED180F1A3008F03ACFE1E0F0E0EC0F97
:102E4000FD1F24E0029FE00DF11D1124208131813E
:102E500042815381AAE0B0E00E94C82D610F711D2C
:102E6000811D911D608371838283938320CF498864
:102E70005A886B887C88812C912C540118CF81143E
:102E80009104A104B10489F4C301B2010E94510A62
:102E900061E070E080E090E00E94CA281D8A1E8AEE
:102EA0001F8A188E312C22242A948D8D9E8DAF8DF1
:102EB000B8A188169906AA06BB06D0F40E940B0A90
:102EC0002D893E894F89588D280F311D411D511D77
:102ED0002D8B3E8B4F8B588F381608F4382E821569
:102EE00008F4282E3FEF831A930AA30AB30A56C0A8
:102EF000C301B20128EE33E040E050E00E94FF2D14
:102F0000BA01A9012AE030E082EE95E00E944A2B46
:102F10006CE282EE95E00E94652A4AE050E0632D63
:102F200082EE95E00E94592B6CE282EE95E00E94C1
:102F3000652A6D897E898F89988DA50194010E94EB
:102F4000FF2DBA01A9012AE030E082EE95E00E944F
:102F50004A2B6CE282EE95E00E94652A4AE050E03E
:102F6000622D82EE95E00E94592B6CE282EE95E094
:102F70000E94A52A4C0C5D1C6E1C7F1C898D9A8DAD
:102F8000AB8DBC8D84159505A605B70520F4498841
:102F90005A886B887C88812C912C540129893A8924
:102FA0004B895C89283E33404105510509F07FCEAD
:102FB000A296E2E10C945C2EACE1B0E0E2EEF7E127
:102FC0000C944A2E0E94A7286B017C0181E00E948C
:102FD000C10A14E703E0198361E0CE0101960E9463
:102FE0001E0C009373050E949C0B6AEF70E080E05A
:102FF00090E00E94CA2880917305833089F482EEA4
:1030000095E00E94A72B892B59F40E94A7286C19E0
:103010007D098E099F096038734C894C9140D8F224
:1030200080917305833009F44FC08FE70E94BA097D
:103030000E94CD098983843511F083E05CC00E9431
:10304000CD0910924605809347050E94CD09209135
:10305000460530914705280F311D309347052093D1
:1030600046050E94CD09809348050E94CD098093B2
:103070004905813110F7F12C0F2D10E080914905A1
:1030800090E0880F991F0817190740F40E94CD0996
:10309000F801E65BFA4F8083F394EECF80E78983F3
:1030A00061E0CE0101960E941E0C83E080937305BF
:1030B0000E949C0B62E370E080E090E00E94CA28CE
:1030C00080917305833011F482E015C08FE70E9470
:1030D000BA090E94CD098983803509F0AECF0FE986
:1030E00015E00E94CD09F80181938F01F5E00A3BBC
:1030F0001F07B9F781E06C96E8E00C94662E80918A
:103100004505992787FD9095A92FB92FFC01319688
:10311000EB30F10508F066C0EC5CFF4F0C94772EA5
:1031200062E778E082EE95E00E94812A82E893E0EF
:103130000E94730C6AE578E082EE95E00E94812A95
:1031400065E378E082EE95E00E94812A6BE078E00A
:1031500082EE95E00E94812A6AEE77E082EE95E0A9
:103160000E94812A6DEB77E082EE95E00E94812A31
:1031700067E977E082EE95E00E94812A63E777E0D5
:1031800082EE95E00E94812A6CE477E082EE95E081
:103190000E94812A82EE95E00E946D2A0E94B10D64
:1031A00021C06FE277E01AC06AE077E017C065EFF0
:1031B00076E014C066ED76E011C062E976E00EC0FC
:1031C0006DE776E00BC068E676E082EE95E00E945F
:1031D000812A62E276E002C06CE076E082EE95E061
:1031E0000E94812A6AE070E080E090E00E94CA2894
:1031F00082EE95E00E94A72B892B29F082EE95E0C4
:103200000E94D42BF5CF0895ACE1B0E0EAE0F9E1FB
:103210000C944A2E909145059F3F09F023C1482FF9
:1032200050E0FA013A97EF36F10508F00FC1E15C82
:10323000FF4F0C94772E61E172E0A0C06DE172E067
:1032400082EE95E00E94932A85E789838BE1EFE97E
:10325000F5E0DE01129601900D928A95E1F76CE19E
:10326000CE0101960E941E0C0E949C0B83E080936D
:10327000730568EC70E080E090E00E94CA288091BD
:103280007305843009F0E2C08FE70E94BA090E94FA
:10329000CD098983853509F0D9C06DEE74E082EEE1
:1032A00095E00E94812A6FEC74E082EE95E00E9426
:1032B000812A61EB74E096C065E372E082EE95E0EE
:1032C0000E94932A89E6898361E0CE0101960E94DB
:1032D0001E0C0E949C0B83E08093730568EC70E0E9
:1032E00080E090E00E94CA2880917305843009F044
:1032F000ADC08FE70E94BA090E94CD0989838E0173
:103300000E5F1F4F7E014DE1E40EF11C0E94CD09BE
:10331000F80181938F01EE15FF05C1F78BE1FE01E6
:103320003296AFE9B5E001900D928A95E1F7898177
:10333000893409F08BC063E974E082EE95E00E9465
:10334000812A65E774E082EE95E00E94812A67E5B4
:1033500074E048C06FE472E082EE95E00E94932A28
:103360008EEF8093450572C08052875080539091B4
:103370004805981708F066C06EE572E082EE95E0A9
:103380000E94932A63C084E18093450560E274E063
:1033900029C085E18093450569EE73E023C086E18D
:1033A0008093450562EB73E01DC087E1809345057E
:1033B00068E673E017C088E18093450567E573E030
:1033C00011C089E18093450563E473E00BC08AE195
:1033D000809345056EE273E005C08BE1809345055F
:1033E00066E073E082EE95E00E94812A2FC06CEEC9
:1033F00072E082EE95E00E94812A8091AD0591E015
:103400001DC066ED72E082EE95E00E94812A8091F7
:10341000AD0592E013C061EC72E082EE95E00E948F
:10342000812A8091AD0594E009C066EA72E082EEDF
:1034300095E00E94812A8091AD0598E089278093CC
:10344000AD058FEF809345050E94521082EE95E006
:103450000E94A72B892B09F45BC182EE95E00E94A4
:10346000D42BF4CF0E945111882309F451C18091CB
:10347000DF04811104C08FEF8093450541C140E016
:1034800050E060E070E080EE94E00E94EE2E40910B
:103490004505042F112707FD1095212F312FF80125
:1034A0003197EB31F10508F01BC1E255FF4F0C9449
:1034B000772E552747FD50952091480530E0241779
:1034C00035070CF40DC18B019C0101501109210934
:1034D0003109003211052105310558F0C090490528
:1034E000EBE4F5E0F12CD12CA8E2EA2E4150510991
:1034F0000FC0FA01E156FA4F61506083D9C0DF0175
:1035000011972C9130E02417350729F0F394329667
:10351000FC10F5CFCBC00E2D10E020E030E00617F8
:1035200017072807390741F42081DA01A156BA4F5D
:1035300011962C93DD24D394E394E8CF6F3F71056B
:103540008105910511F008F0CBC06093B705B0C0BC
:103550006F3F71058105910511F008F0C1C06093BE
:10356000B805A6C06F3F71058105910511F008F0FF
:10357000B7C06093B9059CC02091E0042062203759
:10358000E9F440E050E060E070E081EE94E00E94F9
:10359000EE2E9B01AC01DC01CB010197A109B10921
:1035A0000897A105B10508F0AEC0A4EDB0E30E94F4
:1035B000C82D6A5E7C4A8A46954E24C02636E9F4B8
:1035C00040E050E060E070E081EE94E00E94EE2E7A
:1035D0009B01AC01DC01CB010197A109B10907975F
:1035E000A105B10508F08FC0A8EAB1E60E94C82D78
:1035F000645E7C438E46944E05C06115710581055D
:10360000910579F08B019C010054114E2D493841F0
:103610000138F0EF1F07FAEF2F07F2E03F0708F03D
:103620005FC06093AF057093B0058093B105909330
:10363000B2053EC06F3F71058105910511F008F09C
:103640004FC06093B30534C08B019C010150110938
:10365000210931090F3F11052105310508F040C04E
:103660006093B40525C08B019C01045C19402109BD
:1036700031090D344DE114072105310528F470930B
:10368000B6056093B50514C06115710581059105F6
:1036900021F48FEF8093AE050BC061347105810575
:1036A0009105F0F461506093AE0502C0DD20C1F0D9
:1036B0008091DE0481111AC080917F059091800570
:1036C000A0918105B09182050196A11DB11D809345
:1036D0007F0590938005A0938105B093820506C075
:1036E00060E772E082EE95E00E94932A0E94471103
:1036F0008FEF809345056AE082EE95E00E94A52A4F
:103700000E94521005C061E070E080E090E07ACF46
:103710006C96E8E00C94662E6AE572E082EE95E025
:103720000E94812A62E472E082EE95E00E94812A82
:1037300082EE95E00E94A72B892B31F082EE95E076
:103740000E94D42B0E9404190E94DC17823029F0B9
:10375000833051F46DE072E002C064E272E082EE08
:1037600095E00E94812A08958FEF8093450510927D
:10377000DE040E945210809145058E3F69F082EE72
:1037800095E00E94A72B892BB1F382EE95E00E9471
:10379000D42B0E940419EFCF08950F931F9310911B
:1037A00045051F3F09F0D2C0893409F457C000F520
:1037B000883309F469C058F4803309F477C008F0FD
:1037C00061C08B3109F440C08132B1F1B9C081349C
:1037D00009F487C030F4893309F466C0803461F19C
:1037E000AFC0823409F48EC0863409F448C0A8C042
:1037F000823609F487C078F4883531F128F48235AF
:10380000C1F18335E1F09CC08A3509F494C081365A
:1038100009F467C095C0823761F128F4863679F1E2
:103820008936E1F08DC0883779F08A3709F483C092
:10383000833709F085C003C061E172E015C00E94C2
:10384000820D6EE872E004C00E948B0D68EA72E09F
:1038500082EE95E00E94932A8EEF70C00E947A0655
:103860000E94BF0667EC72E082EE95E00E94932A08
:1038700067C081E00E94DF0660EE72E0F5CF0E9433
:10388000FC105EC080535AC06AEF71E082EE95E092
:103890000E94812A90919E0588E0890F8871977E09
:1038A000892B80939E051AC089E048C067EE71E0BD
:1038B00082EE95E00E94812A8091BF059091C0051B
:1038C000A091C105B091C20520E182278093BF0578
:1038D0009093C005A093C105B093C2051093450510
:1038E0002FC061ED71E082EE95E00E94812A809107
:1038F000BF059091C005A091C105B091C20540E4FB
:10390000842710C060EC71E082EE95E00E94812A6D
:103910008091BF059091C005A091C105B091C205ED
:1039200020E282278093BF059093C005A093C10534
:10393000B093C20502C00E948C1B8FEF8093450597
:10394000809145058E3F09F0D4C0DDC00E94511121
:10395000882309F4D8C08091DF04811104C08FEF5F
:1039600080934505C6C040E050E060E070E080EE26
:1039700094E00E94EE2E00914505112707FD109559
:10398000212F312FF8013197E930F10508F0B4C04B
:10399000E753FF4F0C94772E8B019C010154114E7D
:1039A0002D4938410F37104F2A4F324008F0A4C03C
:1039B00060937B0570937C0580937D0590937E05D5
:1039C00077C060937F057093800580938105909305
:1039D000820581E08093DE046BC06830710581054B
:1039E000910508F089C06093830562C08B019C013A
:1039F00001501109210931090A301105210531054C
:103A000008F07AC06093840553C061EB71E080EEEA
:103A100094E00E94283010E0009799F00E94023054
:103A2000009779F0183130F4E12FF0E0EA58FA4FBE
:103A300087871F5F61EB71E080E090E00E94283093
:103A4000EBCF1831A8F5E12FF0E0EA58FA4F1786CE
:103A50001F5FF7CF653071058105910508F04CC0F7
:103A600060939D0525C08B019C010150110921091E
:103A700031090630110521053105F0F520919E052B
:103A8000287F262B20939E0513C08B019C0101509B
:103A90001109210931090115124C2140310560F548
:103AA00060937705709378058093790590937A05F4
:103AB0008091DE04811113C080917F059091800573
:103AC000A0918105B09182050196A11DB11D809341
:103AD0007F0590938005A0938105B09382050E9495
:103AE00047118FEF809345056AE082EE95E00E94D2
:103AF000A52A0E947F1807C060E772E082EE95E079
:103B00000E94932AECCF1F910F9108958FEF80931D
:103B100045051092DE040E947F18809145058E3F76
:103B200069F082EE95E00E94A72B892BB1F382EE1B
:103B300095E00E94D42B0E94CD1BEFCF6AE070E08D
:103B400080E090E00E94CA2882EE95E00E94A72BB8
:103B5000892B29F082EE95E00E94D42BF5CF0895B1
:103B6000CF93C82F682F82EE95E00E94012C909190
:103B70006A059C2790936A05CF910895A1E0B0E073
:103B8000E4ECFDE10C94502E99830E94B01D9981C4
:103B9000892F0E94B01D2196E2E00C946C2E1F9399
:103BA000CF93DF93182FEB0110926A0565EB70E05D
:103BB00082EE95E00E94590662E670E082EE95E0A2
:103BC0000E945906812F0E94B01DCE010E94BE1D89
:103BD000DF91CF911F91089560916A0582EE95E083
:103BE0000E94012C0895A1E2B0E0E9EFFDE10C9400
:103BF0004C2E7B018A018C3009F452C108F040C080
:103C0000863009F4BCC018F5833009F491C070F413
:103C1000813009F472C0823009F047C26BE170E074
:103C200082E00E94CF1D0FE915E078C0843009F4CE
:103C300087C0853009F039C26091490570E0660F90
:103C4000771F85E00E94CF1D0AE415E086C0893009
:103C500009F4A7C070F4873009F49BC0883009F0DC
:103C600024C261E070E088E00E94CF1D8091D405FD
:103C700022C28A3009F4CAC08B3009F4F1C015C2DF
:103C80008A3609F474C1D8F4873609F439C138F496
:103C9000853609F40DC1863609F41EC106C2883680
:103CA00009F436C1893609F000C261E070E089E6A6
:103CB0000E94CF1D0E947A060E94BF06F4C18D3675
:103CC00009F4D3C138F48B3609F490C18C3609F469
:103CD00099C1EBC18E3609F4DBC1873C09F0E5C11F
:103CE00061E070E087EC0E94CF1D81E00E94B01D72
:103CF0000E94EC1D10926B05E2C169E270E081E068
:103D00000E94CF1D06E715E0F80181918F010E9406
:103D1000B01DF5E00F391F07B9F7CFC1F801819148
:103D20008F010E94B01DF5E00A3B1F07B9F7C5C11E
:103D300061E070E083E00E94CF1D0E94DC17BBC1F0
:103D400061E070E084E00E94CF1D81E00E94B01D20
:103D50000E94EC1D0E940F16B2C18091490590E0AF
:103D6000880F991F98012A5435402817390708F001
:103D7000A4C1F80181918F010E94B01DEECF62E0D5
:103D800070E086E00E94CF1D82E893E00E94BE1D95
:103D900094C161E070E087E00E94CF1D80914805EA
:103DA0008AC186E6898361E0CE0101960E941E0CDD
:103DB0000E949C0B83E08093730568EC70E080E0C8
:103DC00090E00E94CA28809173058430D9F48FE76F
:103DD0000E94BA090E94CD098983863469F460E2A1
:103DE00070E089E00E94CF1D10E20E94CD090E9480
:103DF000B01D1150D1F761C161E070E089E00E940F
:103E0000CF1D51C161E070E089E052C169E170E00D
:103E10008AE00E94CF1D1092BA0520917205809110
:103E2000BF059091C005A091C105B091C2052223A4
:103E300011F0806801C08F778093BF059093C00513
:103E4000A093C105B093C2050AEB15E0F80181917A
:103E50008F010E94B01DF5E0033D1F07B9F72DC18A
:103E600061E270E08BE00E94CF1D8091AA048F3F39
:103E700039F08091AA0491E0980F9093AA0402C0AF
:103E80008091AA040E94B01D10E0812F0E94F115BC
:103E90000E944C090E94BE1D1F5F1031B1F70DC179
:103EA00061E070E08CE00E94CF1D8091D30503C1DA
:103EB00061E070E085E60E94CF1D89E2E816F1041A
:103EC00009F0F8C0D801E6E7F5E08D91819385E02F
:103ED000EF39F807D1F7E7C061E070E086E60E94AD
:103EE000CF1DEBE1EE16F10409F0E4C0D801EFE9D3
:103EF000F5E08D91819385E0EA3BF807D1F7D3C0D7
:103F000061E070E087E60E94CF1D0E94820DCBC069
:103F100061E070E088E60E94CF1D85E789838BE130
:103F2000EFE9F5E0DE01129601900D928A95E1F736
:103F30006CE1CE0101960E941E0C0E949C0B83E056
:103F40008093730560E273E080E090E00E94CA28ED
:103F500080917305843009F0ADC08FE70E94BA09E3
:103F60000E94CD098983853509F0A4C09CC061E019
:103F700070E08AE60E94CF1D89E6898361E0CE0168
:103F800001960E941E0C0E949C0B83E08093730597
:103F900060E273E080E090E00E94CA28809173059F
:103FA000843009F087C08FE70E94BA090E94CD09CA
:103FB00089838E010E5F1F4F7E01EDE1EE0EF11C35
:103FC0000E94CD09F80181938F01EE15FF05C1F71D
:103FD0008BE1FE013296AFE9B5E001900D928A9532
:103FE000E1F78981893409F065C05DC061E070E066
:103FF0008BE60E94CF1DF80180818093D4050E943A
:104000008B0D51C061E070E08CE60E94CF1DF0E2A4
:10401000EF16F10461F487E6898380E2F801DE019E
:10402000129601900D928A95E1F761E203C087E450
:10403000898361E0CE0101960E941E0C0E949C0BB8
:1040400083E0809373056CE474E080E090E00E946C
:10405000CA2880917305843069F58FE70E94BA09F8
:104060000E94CD09873431F51EC061E070E08DE615
:104070000E94CF1D89E1E816F104E1F4D801EAEBD2
:10408000F5E08D91819385E0E33DF807D1F70BC012
:1040900061E070E08EE60E94CF1DF8018081809380
:1040A000D3050E946C0D81E006C061E070E08AECEF
:1040B0000E94CF1D80E00E94B01D0E94EC1DA196C1
:1040C000E6E00C94682EA0E0B0E0E9E6F0E20C94A3
:1040D0004A2ECAECD3E014E606E035E0F32E44E0C5
:1040E000E42E53E0D52E62E0C62E82EE95E00E94CB
:1040F000A72B892B09F49BC082EE95E00E94D42B5C
:10410000282F809335044091340450E04730510506
:1041100060F7FA01EE52FF4F0C94772E853B29F79A
:1041200081E080933404E1CF823609F07DC0C092F3
:104130003404DBCF8093330480933204D092340470
:10414000D4CF9C01332730933104209330049091D5
:104150003204982790933204E0923404C6CF382F6B
:1041600022274091300450913104242B352B309379
:1041700031042093300490913204982790933204B4
:10418000F09234042536310508F4AFCF61E070E0D9
:104190008CEC0E94CF1D81E00E94B01D0E94EC1D9E
:1041A00043C020912E0430912F04F901E653FC4FB7
:1041B000808390913204982790933204C90101962C
:1041C00090932F0480932E04209130043091310479
:1041D0008217930708F489CF0093340486CF809127
:1041E000320482130BC060912E0470912F044AECAC
:1041F00053E0809133040E94F31D0DC062E070E033
:104200008BEC0E94CF1D809133040E94B01D8091E1
:104210006A050E94B01DFE01812F11928A95E9F76F
:1042200010922F0410922E04109234045ECFCDB75A
:10423000DEB7E8E00C94662E81E080936B058091F8
:104240006B05882349F082EE95E00E94A72B892B0D
:10425000B1F30E946320F3CF0895AAE2B0E0E3E354
:10426000F1E20C94482E0E949B286B017C0181E0B6
:104270000E94C10A82EE95E00E94A72B892B29F0AB
:1042800082EE95E00E94D42BF5CF439811E072E6C0
:10429000B72EE9E2AE2E03E00E949B286C197D093F
:1042A0008E099F09693C710581059105D0F11123A3
:1042B000C1F10E949B286B017C01429A80ED97E03E
:1042C0000E94B607B982E6E7F5E0DE0112968A2D74
:1042D00001900D928A95E1F76AE2CE0101960E9463
:1042E0001E0C429880E090E00E94B6070093730590
:1042F0000E949C0B62E370E080E090E00E94CA287C
:1043000080917305843061F4009373058FE70E94F8
:10431000BA090E94CD0911E0823419F410E001C0FD
:1043200011E082E10E94C029892B81F411E00EC0C6
:10433000439A429A82EE95E00E94D42B8D309105EB
:10434000A9F05CF40A9791F04398429882EE95E0C8
:104350000E94A72B892B61F79FCF8332910579F0BB
:104360008234910589F70E941C21EECF62EB71E047
:1043700082EE95E00E94812A0E94861DE5CF0E9470
:104380000F16E2CF8F929F92AF92BF92CF92DF92A1
:10439000EF92FF921F93CF93DF9382E10E94C02997
:1043A000892B09F089C068EC70E080E090E00E9401
:1043B000CA2880E090E00E94B6070E949B284B012B
:1043C0005C016B017C0180ECC80E82E1D81EE11C0F
:1043D000F11C0E949B286C157D058E059F0530F40D
:1043E00082E10E94C029892BA1F364C082E10E946E
:1043F000C029892B09F05EC080ED97E00E94B607C6
:104400000E949B286B017C01D0E0C1E088E4880E0B
:1044100086E2981EA11CB11C11E082E10E94C02915
:10442000892B21F58C149D04AE04BF0430F480ED7B
:1044300097E00E94B607D1E0F0CF0E949B286C194C
:104440007D098E099F09693C71058105910528F355
:104450000E949B286B017C01C12719F080ED97E039
:1044600002C080E090E00E94B607D7CF80E090E0E5
:104470000E94B607DD23B9F08091D30590E0019644
:1044800065E070E00E94EB2D8093D3050E946C0DD7
:104490000E94E6130E948B0D64EF71E080E090E0D3
:1044A0000E94CA2809C080E00E94DF060E94031211
:1044B0000E94820D0E942D21DF91CF911F91FF90CC
:1044C000EF90DF90CF90BF90AF909F908F90089526
:1044D000CF92DF92EF92FF9280E00E941D080E942F
:1044E000F40761E081E10E94542961E080E10E94CB
:1044F000542960E082E10E94542960E088E00E9433
:10450000542961E088E00E948D290E949F0740E0C5
:1045100052EC61E070E082EE95E00E94EF2C0E9488
:10452000E6130E948B0D0E94CB138FEF8093AA0499
:104530000E94090878940E949B286B017C0180915D
:10454000AA048F3F59F40E949B286C197D098E099B
:104550009F09603D77408105910588F380ED97E0E4
:104560000E94B60761E082E10E948D29439A82EEA3
:1045700095E00E94A72B892B29F082EE95E00E94FE
:10458000D42BF5CF6DEF72E082EE95E00E94622AA7
:1045900082E893E00E94730C64E173E082EE95E0A0
:1045A0000E94622A4AE050E068E070E082EE95E006
:1045B0000E94322B62E370E080E090E00E94CA2803
:1045C00082EE95E00E94A72B04970CF182EE95E015
:1045D0000E94D42B82349105D1F482EE95E00E94A2
:1045E000D42B8E34910599F482EE95E00E94D42B61
:1045F0008434910561F482EE95E00E94D42B81977A
:1046000031F480E090E00E94B6070E942D21409195
:104610007705509178056091790570917A05DB01F5
:10462000CA010197A109B1090497A105B10568F470
:104630004093A904433029F440EA56E861E070E071
:1046400004C040E052EC61E070E082EE95E00E9430
:10465000EF2C0E94C221439880E090E00E94B607B0
:104660000E94CB131092C5048091BF0583FF11C037
:1046700080918B05882351F080919205882331F039
:1046800080919905882311F087E001C085E080932F
:10469000C50480E00E94C10A8091C6040E94F50909
:1046A0000E949C0B10923F0410923E0410923D0415
:1046B000F12C8091D4058F15B0F062E370E080E0BA
:1046C00090E00E94CA2880ED97E00E94B60762E35E
:1046D00070E080E090E00E94CA2880E090E00E94B4
:1046E000B607F394E6CF80919E0584FF08C0982F0B
:1046F000987181E0983109F080E00E94BF118FE04D
:104700000E941D08FF90EF90DF90CF900895EF92E8
:10471000FF920F931F93CF93DF938C016EE770E0AE
:1047200082EE95E00E945906E801F12CF0E2EF2EAE
:104730008E0188818D57823048F46DE770E082EEFB
:1047400095E00E94590688818E2588832196F8017C
:10475000608182EE95E00E94012CF394F9E0FF1253
:10476000E7CF6EE770E082EE95E00E945906CDB784
:10477000DEB7E6E00C94682EA9E0B0E0E2ECF3E2EC
:104780000C94502E9091C70491110EC09EEF998306
:104790008A836B8350E0559547954C832D8319860A
:1047A00018861F821E822EC04091CC04842F90E078
:1047B000B4E095958795BA95E1F7242F2F7030E0F6
:1047C0008217930719F18DEF89831B82FE013496BE
:1047D00050E0842F90E0A4E095958795AA95E1F7A5
:1047E000242F2F7030E08217930749F0DC01A35388
:1047F000BB4F8C918193405F5F5F563051F7409380
:10480000CC045A83CE0101960E9487238091C7046D
:1048100090E0019666E070E00E94EB2D8093C70463
:104820002996E2E00C946C2EA0E0B0E0EAE1F4E21C
:104830000C94492E6C016EE770E082EE95E00E94C8
:1048400059068601E12CF12CC0E0D0E030E2B32E15
:10485000F801608183E8860F823078F46DE770E0BC
:1048600082EE95E00E945906F80160816B2570E0A8
:1048700082EE95E00E94590604C082EE95E00E9407
:10488000012CE114F10459F0F80180819E01280FF8
:10489000311DC901C92FDD27C80FD91FDD273FEF03
:1048A000E31AF30A89E0E816F10459F028E0E21669
:1048B000F10421F48C2F8095F60180870F5F1F4F44
:1048C000C7CFCDB7DEB7E9E00C94652EA9E0B0E024
:1048D000ECE6F4E20C94502EE82F362F8091C704BA
:1048E00090E0019664E270E00E94EB2D8093C70493
:1048F00058E9598350E15A83813089F048F0823079
:10490000B9F08330D9F48B8381EF8C833D8319C058
:1049100085E08B8381EF8C832F5F2D8312C08B8387
:1049200081EF8C8384E6489FA00111245D8309C038
:1049300084E08B8381EF8C83ED8303C00E94FC11A4
:1049400004C0CE0101960E9414242996E2E00C9442
:104950006C2EA2E0B0E0EFEAF4E20C94452E182FA2
:10496000762E2A8349830E94A7286B017C018091BF
:10497000DD048090C8049090C904A090CA04B0904F
:10498000CB042A8149818823C1F0D701C601881947
:104990009909AA09BB094C015D0191EE89169EE2B5
:1049A0009906A104B10420F1241708F4422F202F06
:1049B000672D812F0E94662413C0D701C601881974
:1049C0009909AA09BB094C015D0191E3891695E794
:1049D0009906A104B10460F0672D812F0E94BC23C9
:1049E000C092C804D092C904E092CA04F092CB04E9
:1049F0002296EDE00C94612EA2E2B0E0E2E0F5E256
:104A00000C94462E8CE00E94DC0981110DC06CE1F3
:104A100073E082EE95E00E94932A439A80E00E9420
:104A2000C10A0E949C0B439882EE95E00E94A72B3E
:104A3000892B01F182EE95E00E94D42B9091A9047C
:104A4000992319F00E94F913EFCF40913E0450E0F2
:104A50009A012F5F3F4F2F71332760913F0470E021
:104A60002617370709F3FA01E75BFB4F8083209392
:104A70003E04DACF80917305843009F086C00E942D
:104A8000A728611571058105910549F06093B70468
:104A90007093B8048093B9049093BA040CC081E079
:104AA00090E0A0E0B0E08093B7049093B804A093A6
:104AB000B904B093BA048091AD049091AE048160C2
:104AC0009093AE048093AD0483E0809373058FE7E9
:104AD0000E94BA0909E614E00E94CD09F801819309
:104AE0008F01F4E002371F07B9F72091720480911B
:104AF0006904982F922796FF3BC090E492279093E9
:104B00007204982F98739833F1F410E0212F30E05D
:104B100080916904877090E0821793074CF11F5FC2
:104B200020919E05812F90E0FC01E759FB4F24FF67
:104B300004C080810E94DE11E9CF608182EE95E0A1
:104B40000E94012CE3CF8F7399F480916A048093C3
:104B5000B60480916B048093B40480916C048093BC
:104B6000B30480916F0490E09093AC048093AB0405
:104B700080913D04813019F482E080933D0480915E
:104B80003D04833011F410923D040E94A7286B016C
:104B90007C018091AF049091B004A091B104B091D8
:104BA000B2040097A105B105C9F0A7019601281B21
:104BB000390B4A0B5B0BDA01C901883B9B40A1050D
:104BC000B10560F00E940B0A8093B5041092AF0407
:104BD0001092B0041092B1041092B2048091BB0400
:104BE0009091BC04A091BD04B091BE044601570150
:104BF000881A990AAA0ABB0A86E795E00E94370834
:104C000086169706A806B90608F4A8C0C092BB0489
:104C1000D092BC04E092BD04F092BE040E945706FC
:104C20008091AA048830A0F08091BF059091C005C2
:104C3000A091C105B091C2055CE1B695A795979585
:104C400087955A95D1F7892B8A2B8B2B09F09EC11A
:104C50008091AA048F5F8093AA048091B7049091F9
:104C6000B804A091B904B091BA040097A105B105A8
:104C7000F1F0C81AD90AEA0AFB0A86E795E00E9411
:104C800037086C157D058E059F0508F006C18091DB
:104C9000BF0584FD04C080ED97E00E94B607109226
:104CA000B7041092B8041092B9041092BA0490910B
:104CB0007204907C9093720450913E0480913F0462
:104CC00020913D04581709F405C1223009F002C1B2
:104CD000905890937204E0919E05E770F0E0E658DA
:104CE000FC4F6081693008F0DDC0615040E0461340
:104CF000DBC080933F0487E3840F90917204892B7B
:104D0000809372044093400483E080933D04429A70
:104D1000809183059091C504911129C10E94BC0A1C
:104D20008091C6040E94F509E0919E05E770F0E0CD
:104D3000E658FC4F608182E794E00E94D70BE09137
:104D4000C604EF5FE093C604E83109F41CC1F0E04B
:104D5000EA58FA4F8785882309F415C10E94460C4A
:104D6000813069F580919E05887149F18091AD048B
:104D70009091AE04880F991F9093AE048093AD0478
:104D800083E0809373050E949C0B0E94A728609388
:104D9000AF047093B0048093B1049093B204672B76
:104DA000682B692B61F481E090E0A0E0B0E0809393
:104DB000AF049093B004A093B104B093B204809177
:104DC0009E0584FF1FC08091AD049091AE048E7F3C
:104DD0000E946D09182F6091AB048091B6040E9467
:104DE000EF13482F612F8091B50449A30E94EF1360
:104DF0000091D405282F49A16091B3048091B40497
:104E00000E94A92442988091C3048130C1F018F017
:104E10008230B1F1C8C082E10E94C029892B09F01B
:104E2000C2C081E08093C3040E949B286093BF04AA
:104E30007093C0048093C1049093C204B4C082E113
:104E40000E94C029892B31F50E949B28C090BF0485
:104E5000D090C004E090C104F090C2046C197D09A8
:104E60008E099F09693E73408105910508F49BC036
:104E700082E08093C30480ED97E00E94B60793C060
:104E800082E10E94C029892B09F48DC080E090E066
:104E90000E94B6071092C30486C080E090E00E9492
:104EA000B60705CF68E022CF851709F422CF4F5F00
:104EB000242F30E090E0F901EE58FB4FDC01A75BB6
:104EC000BB4F7C917083F901E05CFB4F70830196CE
:104ED0008F710DCF2430B1F42091400481E494E02F
:104EE000A3E7B4E0FC013E2F381B321718F43191D0
:104EF0003D93F9CF87E3820F90917204892B8093C1
:104F0000720402CF8091C304823051F49160909377
:104F10007204439A8E010F5F1F4FF12CB80110C02D
:104F2000439880913D04811103C081E080933D044A
:104F300080913D04833071F784E080933D04EACF93
:104F40008F2D69A37AA30E94F115F80181939193A3
:104F50008F01F39469A17AA1F0E1FF12F1CF809162
:104F60009E0543E754E087700E94BC08D0CE88239A
:104F700009F4D4CE2091C40431E0320F3093C4043C
:104F80002913CCCE0CC01092C604E8CE8091AA049E
:104F9000883009F4439A89E08093AA04DFCE109206
:104FA000C4048150BBCEA296ECE00C94622E8230F9
:104FB000E8F4E82FF0E0EE0FFF1FEB52FA4F718399
:104FC0006083813041F0809169008C7F842B8093D5
:104FD0006900E89A089580916900440F551F440FB5
:104FE000551F837F842B80936900E99A08951F924F
:104FF0000F920FB60F9211242F933F934F935F930D
:105000006F937F938F939F93AF93BF93EF93FF9390
:105010008091D5059091D605892B29F0E091D50591
:10502000F091D6050995FF91EF91BF91AF919F91B6
:105030008F917F916F915F914F913F912F910F9041
:105040000FBE0F901F9018951F920F920FB60F92E0
:1050500011242F933F934F935F936F937F938F937D
:105060009F93AF93BF93EF93FF938091D705909158
:10507000D805892B29F0E091D705F091D80509953D
:10508000FF91EF91BF91AF919F918F917F916F9120
:105090005F914F913F912F910F900FBE0F901F90F6
:1050A00018951F920F920FB60F9211242F933F93D2
:1050B0008F939F93AF93BF938091DA059091DB0517
:1050C000A091DC05B091DD053091D90523E0230FD7
:1050D0002D3720F40196A11DB11D05C026E8230F30
:1050E0000296A11DB11D2093D9058093DA059093F6
:1050F000DB05A093DC05B093DD058091DE05909182
:10510000DF05A091E005B091E1050196A11DB11D5B
:105110008093DE059093DF05A093E005B093E10551
:10512000BF91AF919F918F913F912F910F900FBEA3
:105130000F901F9018952FB7F8946091DA05709131
:10514000DB058091DC059091DD052FBF08953FB709
:10515000F8948091DE059091DF05A091E005B09173
:10516000E10526B5A89B05C02F3F19F00196A11DAA
:10517000B11D3FBF6627782F892F9A2F620F711DAF
:10518000811D911D42E0660F771F881F991F4A9568
:10519000D1F70895CF92DF92EF92FF92CF93DF93F2
:1051A0006B017C010E94A728EB01C114D104E1042A
:1051B000F10479F00E94A7286C1B7D0B683E7340B8
:1051C000A0F381E0C81AD108E108F108C851DC4F0A
:1051D000ECCFDF91CF91FF90EF90DF90CF900895CB
:1051E000789484B5826084BD84B5816084BD85B5C2
:1051F000826085BD85B5816085BDEEE6F0E0808189
:1052000081608083E1E8F0E01082808182608083A9
:10521000808181608083E0E8F0E08081816080832C
:10522000E1EBF0E0808184608083E0EBF0E080815E
:1052300081608083EAE7F0E0808184608083808100
:1052400082608083808181608083808180688083A8
:105250001092C1000895833081F028F4813099F0D4
:105260008230A1F008958630A9F08730B9F08430FB
:10527000D1F4809180008F7D03C0809180008F7772
:1052800080938000089584B58F7702C084B58F7DA8
:1052900084BD08958091B0008F7703C08091B000E5
:1052A0008F7D8093B0000895CF93DF9390E0FC0151
:1052B000ED50F44F2491FC01E95FF34F8491882372
:1052C00049F190E0880F991FFC01E15DF34FA59132
:1052D000B4918B5D934FFC01C591D4919FB761113F
:1052E00008C0F8948C91209582238C938881822326
:1052F0000AC0623051F4F8948C91322F3095832398
:105300008C938881822B888304C0F8948C91822BA3
:105310008C939FBFDF91CF910895A1E0B0E0E3E9C6
:10532000F9E20C944E2E282F30E0F901E152F44FAF
:105330008491F901ED50F44F1491F901E95FF34FB5
:1053400004910023C9F0882321F069830E942B294E
:105350006981E02FF0E0EE0FFF1FEB5DF34FA591A9
:10536000B4919FB7F8948C91611103C0109581237B
:1053700001C0812B8C939FBF2196E4E00C946A2E90
:10538000CF93DF93282F30E0F901E152F44F84915D
:10539000F901ED50F44FD491F901E95FF34FC49155
:1053A000CC2391F081110E942B29EC2FF0E0EE0F1D
:1053B000FF1FE55EF34FA591B4912C912D2381E061
:1053C00090E021F480E002C080E090E0DF91CF9196
:1053D00008958E3008F08E50877020919D0190E4E2
:1053E000299F90011124822B80937C0080917A0068
:1053F000806480937A0080917A0086FDFCCF809152
:1054000078002091790090E0922B0895A0E0B0E020
:10541000ECE0FAE20C944A2E6C017A01EB01E60E04
:10542000F71E00E010E0CE15DF0561F06991D601AE
:10543000ED91FC910190F081E02DC6010995080FD6
:10544000191FF1CFC801CDB7DEB7E8E00C94662E86
:105450006115710589F0DB010D900020E9F7AD01C0
:1054600041505109461B570BDC01ED91FC91028024
:10547000F381E02D0995089580E090E00895EF9282
:10548000FF920F931F93CF93DF938C01FB01C0E03A
:10549000D0E064917F018FEFE81AF80A662361F08B
:1054A000D801ED91FC910190F081E02DC8010995A2
:1054B000C80FD91FF701EDCFCE01CDB7DEB7E6E0BB
:1054C0000C94682E0E94282A0895DC01ED91FC912D
:1054D0000190F081E02D099508950F931F93CF93CC
:1054E000DF93EC016DE00E94652A8C016AE0CE0139
:1054F0000E94652A800F911FDF91CF911F910F911C
:1055000008950F931F93CF93DF93EC010E943F2ADE
:105510008C01CE010E946D2A800F911FDF91CF91E7
:105520001F910F9108950F931F93CF93DF93EC0179
:105530000E94282A8C01CE010E946D2A800F911FA3
:10554000DF91CF911F910F9108950F931F93CF93E8
:10555000DF93EC010E94652A8C01CE010E946D2A26
:10556000800F911FDF91CF911F910F910895A1E2BC
:10557000B0E0EDEBFAE20C94462E7C01C42EE52F50
:10558000CB01D22E19A221E02D1510F02AE0D22E47
:105590008E010F5D1F4F8D2C912CA12CB12C6C2DE9
:1055A0007E2FA50194010E94FF2D8C2DD29E801983
:1055B0001124015011098A3010F4805D01C0895C0A
:1055C000F8018083211531054105510521F0C22ED6
:1055D000E32FCA01E4CFB801C7010E94282AA1968F
:1055E000ECE00C94622EA0E0B0E0E9EFFAE20C945B
:1055F0004A2EEC016A017B012115310541F4E88155
:10560000F9810190F081E02D642F09951DC02A30A9
:105610003105A9F477FF12C06DE20E94652A8C0162
:1056200044275527BA014C195D096E097F092AE004
:10563000CE010E94B72A800F911F06C02AE0B70151
:10564000A601CE010E94B72ACDB7DEB7E8E00C94E0
:10565000662E9A01AB01662757FD6095762F0E9452
:10566000F32A08950F931F93CF93DF93EC019A01D0
:10567000AB01662757FD6095762F0E94F32A8C01B7
:10568000CE010E946D2A800F911FDF91CF911F9153
:105690000F9108952115310549F4DC01ED91FC913C
:1056A0000190F081E02D642F099508950E94B72A9A
:1056B00008959A01462F50E060E070E00E944A2B66
:1056C00008959A01AB0160E070E00E944A2B0895B2
:1056D0000F931F93CF93DF93EC010E944A2B8C0111
:1056E000CE010E946D2A800F911FDF91CF911F91F3
:1056F0000F9108950F931F93CF93DF93EC019A01BD
:10570000AB0160E070E00E944A2B8C01CE010E9448
:105710006D2A800F911FDF91CF911F910F910895F6
:105720000F931F93CF93DF93EC019A01462F50E024
:1057300060E070E00E944A2B8C01CE010E946D2A2D
:10574000800F911FDF91CF911F910F910895FC0160
:1057500024853585F901E05CFF4F80819181F90155
:10576000EE5BFF4F20813181821B930B8F73992752
:105770000895FC0184859585FC01E05CFF4F408124
:105780005181FC01EE5BFF4F2081318142175307AD
:1057900041F00190F081E02DE80FF91F808190E049
:1057A00008958FEF9FEF0895FC0184859585FC0196
:1057B000E05CFF4F40815181FC01EE5BFF4F208197
:1057C00031814217530779F0A081B181A80FB91F29
:1057D0008C91208131812F5F3F4F2F73332731838D
:1057E000208390E008958FEF9FEF0895FC0181A141
:1057F000882329F0A489B5898C9186FFFBCF11A25B
:105800000895CF93DF93FC0126853785D901A05CED
:10581000BF4F8D919C91119701968F739927E90144
:10582000CE5BDF4F4881598184179507D9F30D90DE
:10583000BC91A02DA20FB31F6C93A685B785A05C69
:10584000BF4F11969C938E93A689B7892C9181E0C6
:1058500090E0078C02C0880F991F0A94E2F7282B6A
:105860002C9381E081A30488F589E02D80818064F8
:10587000808381E090E0DF91CF91089508951F9299
:105880000F920FB60F9211242F933F934F938F9344
:105890009F93EF93FF938091C00082FD1CC04091C5
:1058A000C600809188069091890601968F7399278A
:1058B00020918A0630918B068217930771F0E09150
:1058C0008806F0918906E85BF94F4083909389063A
:1058D0008093880602C08091C600FF91EF919F914E
:1058E0008F914F913F912F910F900FBE0F901F906E
:1058F000189582EE95E00E94A72B892B11F00E944B
:105900003E2C08951F920F920FB60F9211242F93E1
:105910003F938F939F93EF93FF9320914406309191
:10592000450680914606909147062817390731F4BD
:105930008091C1008F7D8093C10014C0E091460624
:10594000F0914706EC5FF94F2081809146069091D7
:10595000470601968F7399279093470680934606D2
:105960002093C600FF91EF919F918F913F912F91CE
:105970000F900FBE0F901F901895A0E0B0E0E3ECE1
:10598000FCE20C94462EFC011382128288EE93E016
:10599000A0E0B0E084839583A683B7838CEB93E08B
:1059A000918380837587648757874687318B208BE7
:1059B000138B028BF58AE48AD78AC68AB18EA08EB1
:1059C000938E828E8F85848F8889858F8989868F33
:1059D0008A89878F8B8980A3ECE00C94622ECF920A
:1059E000DF92EF92FF92CF93DF93EC016A017B018C
:1059F000411581EE580761057105F9F0EC89FD89C3
:105A000081E090E008A002C0880F991F0A94E2F795
:105A1000808360E079E08DE390E0A70196010E9429
:105A2000FF2D215031094109510956954795379568
:105A30002795211580E1380798F0EC89FD891082BF
:105A400060E874E88EE190E0A70196010E94FF2DC6
:105A500021503109410951095695479537952795A8
:105A6000E889F9893083EA89FB89208319A2EE89C4
:105A7000FF89408181E090E09C010C8C02C0220FE4
:105A8000331F0A94E2F7422B4083EE89FF8940815D
:105A90009C010D8C02C0220F331F0A94E2F7422BA7
:105AA0004083EE89FF8940819C010E8C02C0220F49
:105AB000331F0A94E2F7422B4083EE89FF8920814D
:105AC0000F8C02C0880F991F0A94E2F780958223F9
:105AD0008083DF91CF91FF90EF90DF90CF9008957A
:105AE0008F929F92AF92BF92CF92DF92EF92FF92EE
:105AF0000F931F9381E08F9385E08F9387E08F93BF
:105B000083E08F9384E08F93E6EC8E2E912CF2EC61
:105B1000AF2EB12CA1ECCA2ED12CB0ECEB2EF12C77
:105B200004EC10E025EC30E044E056E068E476E078
:105B300082EE95E00E94BD2C0F900F900F900F9079
:105B40000F901F910F91FF90EF90DF90CF90BF903B
:105B5000AF909F908F9008950E94F0280E94682235
:105B6000C9E7DCE20E94FC242097E1F30E94792C33
:105B7000F9CFA29FB001B39FC001A39F700D811DFB
:105B80001124911DB29F700D811D1124911D089546
:105B90000E94B92DA59F900DB49F900DA49F800DDC
:105BA000911D11240895B7FF0C94C82D0E94C82D93
:105BB000821B930B0895DB018F939F930E94C82D46
:105BC000BF91AF91A29F800D911DA39F900DB29F99
:105BD000900D1124089597FB072E16F4009407D01A
:105BE00077FD09D00E947D2E07FC05D03EF49095EC
:105BF00081959F4F0895709561957F4F0895A1E21B
:105C00001A2EAA1BBB1BFD010DC0AA1FBB1FEE1F36
:105C1000FF1FA217B307E407F50720F0A21BB30B81
:105C2000E40BF50B661F771F881F991F1A9469F7FD
:105C300060957095809590959B01AC01BD01CF0159
:105C40000895052E97FB1EF400940E94382E57FDF0
:105C500007D00E94FF2D07FC03D04EF40C94382E81
:105C600050954095309521953F4F4F4F5F4F089588
:105C700090958095709561957F4F8F4F9F4F0895B8
:105C80002F923F924F925F926F927F928F929F924C
:105C9000AF92BF92CF92DF92EF92FF920F931F933A
:105CA000CF93DF93CDB7DEB7CA1BDB0B0FB6F894EB
:105CB000DEBF0FBECDBF09942A88398848885F842B
:105CC0006E847D848C849B84AA84B984C884DF809C
:105CD000EE80FD800C811B81AA81B981CE0FD11D80
:105CE0000FB6F894DEBF0FBECDBFED010895EE0FE5
:105CF000FF1F0590F491E02D0994AA1BBB1B51E1F5
:105D000007C0AA1FBB1FA617B70710F0A61BB70B2B
:105D1000881F991F5A95A9F780959095BC01CD01D0
:105D200008958F929F92AF92BF92CF92DF92EF929F
:105D3000FF92CF93DF93EC01688179818A819B8107
:105D4000611571058105910521F464E279ED8BE51A
:105D500097E02DE133EF41E050E00E94212E490110
:105D60005A019B01AC01A7EAB1E40E94C82D6B0166
:105D70007C01ACEEB4EFA50194010E94D62DC60EB5
:105D8000D71EE81EF91EF7FE06C081E0C81AD1082A
:105D9000E10880E8F80AC882D982EA82FB82C7015A
:105DA000B6019F77DF91CF91FF90EF90DF90CF907A
:105DB000BF90AF909F908F9008950E94912E08956C
:105DC00086E091E00E94912E089560930601709301
:105DD0000701809308019093090108952F923F9243
:105DE0005F926F927F928F929F92AF92BF92CF926B
:105DF000DF92EF92FF920F931F93CF93DF938B016C
:105E0000EA016115710521F0DB018C9311969C93D9
:105E1000209739F09E01225031092332310508F0D4
:105E2000D8C07C016701BFEFCB1ADB0A5601F7012E
:105E30006080862D90E00E942030892B11F0760141
:105E4000F1CFFDE26F120AC0570182E0A80EB11C2B
:105E5000D70111966C90772473940BC0BBE26B1240
:105E600007C05701E2E0AE0EB11CD70111966C904D
:105E7000712CCE018F7E892B89F4B0E36B1237C071
:105E8000F50180818F7D8835D1F46180F2E0AF0E1D
:105E9000B11C872D8260782EC0E1D0E0CA30D105D8
:105EA00051F1C031D10521F0C830D10599F409C0B4
:105EB000CC24CA94DC2CEC2CAFE0FA2E22C0209724
:105EC00069F7C8E0D0E0CC24CA94DC2CEC2CFFE1CC
:105ED000FF2E17C06FEF7FEFCB019E01442737FDE8
:105EE0004095542F0E94FF2D69017A010AC0209726
:105EF000A9F6CAE0D0E0E9E9CE2EDC2CEC2CE9E1F1
:105F0000FE2EF50160E020E030E0A9014E01AA2458
:105F100097FCA094BA2C1F0170ED572E560CA9E0E7
:105F2000A51570F48FEB860D8A3118F499EC592E73
:105F300006C08FE9860D8A3148F589EA582E560C3D
:105F4000852D90E08C179D070CF56F3FD9F0C21698
:105F5000D306E406F50698F0C501B4010E94DB2DD6
:105F60009B01AC01852D90E0A0E0B0E0280F391F27
:105F70004A1F5B1F281739074A075B0710F46FEFAA
:105F800001C061E03196D1016C90C5CF01151105BA
:105F900051F0662311F0319703C071FE04C03297AF
:105FA000D801ED93FC9370FE07C050954095309555
:105FB00021953F4F4F4F5F4F67FF10C082E290E047
:105FC00090938D0680938C066FEF7FEF8FEF9FEF9E
:105FD00007C060E070E080E090E002C0B901CA0153
:105FE000DF91CF911F910F91FF90EF90DF90CF90B5
:105FF000BF90AF909F908F907F906F905F903F90F9
:106000002F900895FC0188279927E8942191203248
:10601000E9F3293010F02E30C8F32B3241F02D3245
:1060200039F4689404C00E945430820F911D21916C
:1060300020532A30C0F31EF4909581959F4F089508
:10604000911150C0803219F089508550D0F70895D1
:1060500048EC53E00E942D300895FA01A191B081DF
:10606000009719F41097E1F0CD01DC01CD010D90FE
:10607000002011F4C00113C0FB012191222319F06B
:106080002015D9F7F3CFFB012191201519F41E92A9
:10609000119606C02223C1F70D900020A1F7D00170
:1060A000FA01A193B08308957AE0979F902D879F7E
:1060B000802D910D11240895F999FECF92BD81BDD7
:1060C000F89A992780B50895262FF999FECF1FBA1F
:1060D00092BD81BD20BD0FB6F894FA9AF99A0FBE11
:0E60E00001960895992788270895F894FFCF18
:1060EE0000008E06200001000000FF0002000200EA
:1060FE000200020002000200020002000200020082
:10610E0002000200020002000200028025000005CB
:10611E00400AA1204EA50020244EA52C2330C012EB
:10612E0000001A400AA1204EA5001B1E27522C2348
:10613E00308025000005400AA1204EA50020244EE7
:10614E00A52C2330004B000006400AD0009D4900CC
:10615E007B289D492C233000E1000005400A4501B3
:10616E00D7DC03B81E0EBF00232E48E801008A407C
:10617E000A6001555502AD1E20000023C801545877
:10618E002074696D656F75742100596573004E6FCB
:10619E00002C00386368004E2F41002C205B005D00
:1061AE002028002900486F70206368616E6E656C50
:1061BE00200020402000456E746572696E67206174
:1061CE0064617074697665206368616E6E656C20BB
:1061DE0073656C656374696F6E2C207069636B698F
:1061EE006E673A007363616E6E6572206D6F6465E3
:1061FE00004E4F5420454E41424C45440053656E6F
:10620E0064696E672073657474696E677320746F4A
:10621E002052580A00526573657474696E67207354
:10622E00657474696E6773206F6E2052580A004150
:10623E00626F727465642065646974730A00696EB6
:10624E0076616C69642073656C656374696F6E004A
:10625E000D0A496E76616C696420696E70757420E2
:10626E002D20646973636172646564210700536550
:10627E007474696E677320736176656420746F2021
:10628E00454550524F4D0A005265766572746564ED
:10629E002073657474696E67732066726F6D204526
:1062AE004550524F4D0A004C6F6164656420666123
:1062BE0063746F72792064656661756C74730A001D
:1062CE004B657920616E64206368616E6E656C73D8
:1062DE002072616E646F6D697A65640A004F706535
:1062EE006E4C52536E6720545820737461727469E9
:1062FE006E672000206F6E20485720006D6F64750A
:10630E006C65206C6F636B65643F00342B34003812
:10631E0000382B340031320031322B34003136004C
:10632E0050504D0052535349005344410053434C77
:10633E0000525844005458440041494E004C4245C6
:10634E0045500053504B54524D0053425553005339
:10635E00554D44004C4C494E440000070B0C101197
:10636E001500B7012B032F033103350338033D030B
:10637E00B7014003440349034D0351035503590329
:10638E005D0363036A036F0374038D028D028D0236
:10639E008D02160A1322312900000000012C062A54
:0863AE00A72BD42BB92BF62B11
:00000001FF
